:100000000C942A000C9445000C9445000C94450077
:100010000C9445000C9445000C9445000C9445004C
:100020000C9445000C9445000C9445000C9445003C
:100030000C9445000C9445000C9445000C9445002C
:100040000C9445000C9445000C9445000C9445001C
:100050000C94450011241FBECFE5D8E0DEBFCDBF14
:1000600010E0A0E6B0E0E2EFF7E002C005900D92EC
:10007000A838B107D9F710E0A8E8B0E001C01D9298
:10008000A838B107E1F70C9447030C9400000097DF
:1000900011F00197F1F70895DD9ADD9808951BBAE4
:1000A0000E944C0081E08BBB0E944C0088EE93E0E4
:1000B0000E94470008951BBA0E944C0082E08BBB4F
:1000C0000E944C0088EE93E00E94470008950F9331
:1000D0001F93CF93182FC62F042F1BBA0E944C00DA
:1000E00088E0113029F0C13031F0013041F406C010
:1000F0008CE0C130D1F78260013009F481608BBBA4
:100100000E944C0084E690E00E944700CF911F912E
:100110000F9108951F93182F82958F7088608BBB65
:100120000E944C001F701BBB0E944C0084E690E0B4
:100130000E9447001F9108951F93182F82958F707A
:1001400080618BBB0E944C00812F8F7080618BBBC4
:100150000E944C0084E690E00E9447001F910895A1
:10016000CF93DF93EC018881882361F089910E940D
:100170009C008881882331F089910E949C008881AD
:100180008823A1F7DF91CF9108951F93CF93182F64
:10019000C0E802C080E304C0812F8C23D9F381E33F
:1001A0000E949C00C695C1F7CF911F910895CF93EF
:1001B000982F82958F70805D8A3308F0895F9F70D9
:1001C000C92FC05DCA3308F0C95F0E949C008C2F04
:1001D0000E949C00CF9108950F931F93CF93DF93BC
:1001E000EC0184369105D8F46AE070E00E94C20305
:1001F0008B01862F805D0E949C00C801880F991F8B
:10020000880F991F880F991F800F911F800F911FD2
:10021000C81BD90B8C2F805D0E949C0004C080E617
:1002200090E00E94B000DF91CF911F910F9108954F
:10023000EF92FF920F931F93CF93DF93EC0183E034
:10024000C83ED80788F544E6E42EF12CCE01B7016C
:100250000E94C2038B01862F805D0E949C000E9D30
:10026000C0010F9D900D1E9D900D1124C81BD90B30
:10027000CE016AE070E00E94C2038B01862F805D90
:100280000E949C00C801880F991F880F991F880F32
:10029000991F800F911F800F911FC81BD90B8C2FA6
:1002A000805D0E949C0004C080E690E00E94B00047
:1002B000DF91CF911F910F91FF90EF900895CF9212
:1002C000DF92EF92FF920F931F937C01E0E1CE2E1D
:1002D000E7E2DE2EB6010E94C2038B01862F805D0D
:1002E0000E949C000C9DC0010D9D900D1C9D900DC9
:1002F0001124E81AF90A78EEC72E73E0D72EC70149
:10030000B6010E94C2038B01862F805D0E949C0073
:100310000C9DC0010D9D900D1C9D900D1124E81A9F
:10032000F90A64E6C62ED12CC701B6010E94C203A9
:100330008B01862F805D0E949C000C9DC0010D9D4D
:10034000900D1C9D900D1124E81AF90AC7016AE06E
:1003500070E00E94C2038B01862F805D0E949C008A
:10036000C801880F991F880F991F880F991F800F48
:10037000911F800F911FE81AF90A8E2D805D0E944F
:100380009C001F910F91FF90EF90DF90CF90089508
:10039000AF92BF92CF92DF92EF92FF920F931F9393
:1003A000CF93DF937B018C01A12C9AECB92E9AE9B3
:1003B000C92E9BE3D92EC801B701A60195010E9461
:1003C000D603E901822F805D0E949C00CE01AA27FE
:1003D000BB27BC01CD01A60195010E94A303DC014E
:1003E000CB01E81AF90A0A0B1B0BA12C81EEB82EDF
:1003F00085EFC82E85E0D82EC801B701A60195016A
:100400000E94D603E901822F805D0E949C00CE01EC
:10041000AA27BB27BC01CD01A60195010E94A30319
:10042000DC01CB01E81AF90A0A0B1B0BC0E8AC2E61
:10043000C6E9BC2EC8E9CC2ED12CC801B701A60153
:1004400095010E94D603E901822F805D0E949C00E5
:10045000CE01AA27BB27BC01CD01A60195010E94B0
:10046000A303DC01CB01E81AF90A0A0B1B0BB0E469
:10047000AB2EB2E4BB2EBFE0CB2ED12CC801B7010E
:10048000A60195010E94D603E901822F805D0E949A
:100490009C00CE01AA27BB27BC01CD01A601950176
:1004A0000E94A303DC01CB01E81AF90A0A0B1B0B1B
:1004B000A0EAAA2EA6E8BA2EA1E0CA2ED12CC80125
:1004C000B701A60195010E94D603E901822F805D44
:1004D0000E949C00CE01AA27BB27BC01CD01A6012A
:1004E00095010E94A303DC01CB01E81AF90A0A0B6B
:1004F0001B0BC801B70120E137E240E050E00E9449
:10050000D603E901822F805D0E949C0080E197E282
:10051000C89F9001C99F300DD89F300D1124C9018B
:10052000AA27BB27E81AF90A0A0B1B0BC801B70157
:1005300028EE33E040E050E00E94D603E901822F2C
:10054000805D0E949C0088EE93E0C89F9001C99F47
:10055000300DD89F300D1124C901AA27BB27E81AF6
:10056000F90A0A0B1B0BC801B70124E630E040E092
:1005700050E00E94D603E901822F805D0E949C001A
:1005800084E690E0C89F9001C99F300DD89F300D40
:100590001124C901AA27BB27E81AF90A0A0B1B0B69
:1005A000C801B7012AE030E040E050E00E94D603E5
:1005B000E901822F805D0E949C00CE01880F991F67
:1005C000880F991F880F991F8C0F9D1F8C0F9D1FDF
:1005D000AA27BB27E81AF90A0A0B1B0B8E2D805D90
:1005E0000E949C00DF91CF911F910F91FF90EF909F
:1005F000DF90CF90BF90AF9008951F938FEF8ABB8D
:1006000080E197E20E94470013E01BBB0E944C0070
:1006100084EF91E00E9447001BBB0E944C0084E6DF
:1006200090E00E9447001BBB0E944C0084E690E0D3
:100630000E94470012E01BBB0E944C0084E690E041
:100640000E9447001BBB0E944C0088E08BBB0E94AD
:100650004C0084E690E00E9447001BBA0E944C00C8
:100660008FE08BBB0E944C0084E690E00E94470024
:100670001BBA0E944C0086E08BBB0E944C0084E6B3
:1006800090E00E9447000E944F001F910895CFE123
:10069000D8E0DEBFCDBF0E94FD0240E0642F81E0C4
:1006A0000E94670080E40E948A000E945B0084E64A
:1006B00090E00E94B00080E40E948A0086E790E00B
:1006C0000E94B00080E090E00C94F8039C01832F1E
:1006D000992780BD29B988E18AB98EE880BD08953F
:1006E0005F9BFECF8CB1992708955D9BFECF8CB99F
:1006F0000895CF93982F82958F70805D8A3308F08C
:10070000895F9F70C92FC05DCA3308F0C95F0E941E
:1007100075038C2F0E947503CF910895CF93DF93BB
:10072000EC018881882361F089910E94750388819A
:10073000882331F089910E94750388818823A1F76D
:10074000DF91CF910895629FD001739FF001829F46
:10075000E00DF11D649FE00DF11D929FF00D839F50
:10076000F00D749FF00D659FF00D9927729FB00DED
:10077000E11DF91F639FB00DE11DF91FBD01CF0100
:1007800011240895AA1BBB1B51E107C0AA1FBB1F60
:10079000A617B70710F0A61BB70B881F991F5A950D
:1007A000A9F780959095BC01CD010895A1E21A2E7C
:1007B000AA1BBB1BFD010DC0AA1FBB1FEE1FFF1F05
:1007C000A217B307E407F50720F0A21BB30BE40B55
:1007D000F50B661F771F881F991F1A9469F760959C
:1007E0007095809590959B01AC01BD01CF01089556
:0207F000FFCF39
:1007F200457272004841484120796F7520686176E0
:100802006520746F200074616B65206D65206170D6
:08081200617274203A29000014
:00000001FF
